:10000000B6010C29A501A400B7172730A3001030B2
:1000100015200330A300E8301520A301643015201B
:10002000A3010A30152024082028A2002508A100D9
:100030002408A000D5202008031DB713B71B080013
:10004000303EA7000711871007108316071187108D
:100050000710F030860583122708B6184D283A306D
:10006000A1009830AA203330A60062201330A100EE
:100070008830AA2062206430A92062206430A92040
:100080002230A600622028304C200C304C20063054
:100090004C20B61427084D283614A600361C5B28C1
:1000A0008710033C031C602860200730A100D0307B
:1000B000AA20031408003614FE3C031907298714EC
:1000C000A60E361C36100715F030860526080F39A7
:1000D00086040711A60E361862283230A9200314B0
:1000E0000800A000A00DA00DA00D3830A0058130A3
:1000F00020049F000030A1003230AA201F151F19D4
:100100007F281E08A10083161E08072903178D00EB
:1001100083168C130C1483120C08072903178C0008
:1001200083168C130C1555308D00AA308D008C145D
:100130008C1898280C110729A301A200FF30A207F0
:10014000031CA307031C07290330A100E730AA20E2
:100150009E28A101FC3EA000A109031CB528FF3088
:100160000000A0070318B028A0076400A10FAF2863
:100170000800A2000230C528A2000330C528A20052
:100180000130C528A2000430C528A8002308210298
:10019000031DCC2822082002043003180130031963
:1001A00002302805031DFF3007291030A600A501E5
:1001B000A401210DA40DA50D2208A4022308031CEF
:1001C000230FA5020318EB282208A407230803180D
:1001D000230FA5070310A00DA10DA60BD9282008F9
:1001E00007291030A800A101A001A70CA60C031C30
:1001F000FF282208A00723080318230FA107A10C3A
:10020000A00CA50CA40CA80BF5282408072983131F
:1002100003138312640008008316DF3085008230E8
:100220009F0070308600811387018312850186014B
:1002300087018A11F929861783168613FE308312E7
:100240008A01212001308A01212048308A012120A1
:1002500069308A01212020308A01212047308A011B
:10026000212075308A01212079308A0121207330C4
:100270008A01212021308A01212020308A01212079
:1002800072308A01212065308A01212076308A016E
:10029000212031308A0121202E308A012120303066
:1002A0008A0121200330A300E8308A019D20FE301E
:1002B0008A012120C0308A01212050308A0121206A
:1002C00072308A0121206F308A01212064308A0136
:1002D000212075308A01212063308A012120653078
:1002E0008A01212064308A01212020308A012120C6
:1002F00062308A01212079308A01212020308A0150
:10030000212041308A0121204F308A0121205230A2
:100310008A01212063308A0121200330A300E830C4
:100320008A019D20080003308A017120BC00210849
:10033000BD000A308A019C20080002308A01712029
:10034000C2002108C3000A308A019C200800013045
:100350008A017120C6002108C7000A308A019C204A
:10036000080000308A017120CA002108CB000A3041
:100370008A019C200800FE308A012120C0308A01B9
:10038000212052308A01212065308A0121206D30E0
:100390008A01212061308A01212069308A012120CF
:1003A0006E308A0121205508A50054088A010320D7
:1003B00030308A01212073308A0121203A308A01AD
:1003C00021203F08A5003E088A01032063308A01EE
:1003D000212020308A01212020308A012120203054
:1003E0008A01212020308A01212020308A01212009
:1003F00008000713831607138312071283160712C8
:100400008312871183168711831285128316851232
:1004100083128A011B213E30E2003E30E3003E3071
:10042000E4003E30E50064308A019C2064008A11BB
:10043000061F132A861383168613FE3083128A0141
:10044000212001308A01212042308A0121203A30C6
:100450008A01212054308A01212069308A0121201B
:1004600072308A01212065308A01212020308A01E2
:10047000212068308A01212065308A0121206130E5
:100480008A01212074308A01212020308A01212014
:1004900063308A0121206F308A0121206E308A0169
:1004A000212074308A012120FE308A012120C030B1
:1004B0008A01212059308A0121203A308A012120E5
:1004C0004D308A0121206F308A01212074308A0149
:1004D00021206F308A01212072308A0121202030B2
:1004E0008A01212064308A01212072308A01212072
:1004F00065308A01212073308A01212073308A01FE
:1005000021200130A3002C308A019D2064008A1133
:10051000061E902A64008A15861E46288A01862AAD
:1005200064308A019C2064008A11061E902A0530DE
:100530008A018620DE00DF0109308A018620D8008A
:10054000D9010A308A018620DA00DB010B308A01EA
:100550008620DC00DD01E001E101FE308A0121207E
:1005600001308A01212054308A01212065308A011E
:1005700021206D308A01212070308A0121205F08FE
:10058000A5005E088A0103203A308A01212059081B
:10059000A50058088A0103203A308A0121205B080F
:1005A000A5005A088A0103203A308A0121205D08FB
:1005B000A5005C088A010320FE308A012120C0309A
:1005C0008A01212043308A01212068308A012120BC
:1005D00061308A0121206E308A01212067308A0132
:1005E000212065308A0121203F308A0121202030DE
:1005F0008A01212052308A0121203A308A012120AB
:100600004E308A01212020308A01212042308A0187
:1006100021203A308A01212059308A012120C83016
:100620008A019C2064008A11061E1C2B64008A111A
:10063000061FAE2D8A01122B64308A019C206400B3
:100640008A11061E1C2BFE308A01212001308A01EE
:10065000212041308A01212020308A01212054307C
:100660008A01212065308A0121206D308A012120F4
:1006700070308A0121202E308A01212020308A0109
:10068000212073308A01212065308A0121207430B5
:100690008A0121203D308A0121205F08A5005E08E3
:1006A0008A010320FE308A012120C0308A012120E6
:1006B00052308A0121203A308A0121204E308A01AD
:1006C000212065308A01212078308A012120743070
:1006D0008A01212020308A01212059308A012120DD
:1006E0003A308A01212044308A0121206E308A016B
:1006F000212020308A01212042308A0121203A30F5
:100700008A01212055308A01212070308A01212060
:10071000C8308A019C2064008A11061E992B64004F
:100720008A11861EAC2B64008A11061FC22B8A0117
:100730008B2BDE0A0319DF0A5E08A0005F08A10008
:10074000A30150308A01C2208A11031DAA2B503008
:10075000DE00DF018A01232B0130DE020030031CA2
:10076000013EDF025E08A0005F08A100A3010A307D
:100770008A01BF208A11031DC02B0A30DE00DF0171
:100780008A01232B32308A019C2064008A11061FC3
:10079000C22BFE308A01212001308A012120423003
:1007A0008A01212020308A01212054308A01212011
:1007B00065308A0121206D308A01212070308A0144
:1007C00021202E308A01212020308A0121207330FF
:1007D0008A01212065308A01212074308A0121207C
:1007E0003D308A0121205908A50058088A010320BC
:1007F000FE308A012120C0308A01212052308A0136
:1008000021203A308A0121204E308A012120653092
:100810008A01212078308A01212074308A01212028
:1008200020308A01212059308A0121203A308A0162
:10083000212044308A0121206E308A01212020307D
:100840008A01212042308A0121203A308A01212068
:1008500055308A01212070308A012120C8308A0158
:100860009C2064008A11061E3F2C64008A11861E9B
:10087000522C64008A11061F682C8A01312CD80A78
:100880000319D90A5808A0005908A100A301503043
:100890008A01C2208A11031D502C5030D800D90182
:1008A0008A01C92B0130D8020030031C013ED90255
:1008B0005808A0005908A100A3010A308A01BF20EE
:1008C0008A11031D662C0A30D800D9018A01C92B70
:1008D00032308A019C2064008A11061F682CFE3089
:1008E0008A01212001308A01212043308A01212000
:1008F00020308A01212054308A01212065308A016C
:1009000021206D308A01212070308A0121202E3073
:100910008A01212020308A01212073308A01212080
:1009200065308A01212074308A0121203D308A01FE
:1009300021205B08A5005A088A010320FE308A01A5
:100940002120C0308A01212052308A0121203A30F2
:100950008A0121204E308A01212065308A01212020
:1009600078308A01212074308A01212020308A01C8
:10097000212059308A0121203A308A012120443037
:100980008A0121206E308A01212020308A01212015
:1009900042308A0121203A308A01212055308A01D3
:1009A000212070308A012120C8308A019C206400F7
:1009B0008A11061EE52C64008A11861EF82C64003C
:1009C0008A11061F0E2D8A01D72CDA0A0319DB0AB9
:1009D0005A08A0005B08A100A30150308A01C22080
:1009E0008A11031DF62C5030DA00DB018A016F2CCE
:1009F0000130DA020030031C013EDB025A08A0007D
:100A00005B08A100A3010A308A01BF208A11031DDF
:100A10000C2D0A30DA00DB018A016F2C32308A019A
:100A20009C2064008A11061F0E2DFE308A012120B1
:100A300001308A01212044308A01212020308A019E
:100A4000212054308A01212065308A0121206D3017
:100A50008A01212070308A0121202E308A01212034
:100A600020308A01212073308A01212065308A01DB
:100A7000212074308A0121203D308A0121205D0827
:100A8000A5005C088A010320FE308A012120C030C5
:100A90008A01212052308A0121203A308A01212006
:100AA00047308A0121206F308A01212020308A01BD
:100AB000212059308A0121203A308A0121204430F6
:100AC0008A0121206E308A01212020308A012120D4
:100AD00042308A0121203A308A01212055308A0192
:100AE000212070308A012120C8308A019C206400B6
:100AF0008A11061E852D64008A11861E982D6400B9
:100B00008A11061FAE2D8A01772DDC0A0319DD0A32
:100B10005C08A0005D08A100A30150308A01C2203A
:100B20008A11031D962D5030DC00DD018A01152D40
:100B30000130DC020030031C013EDD025C08A00035
:100B40005D08A100A3010A308A01BF208A11031D9C
:100B5000AC2D0A30DC00DD018A01152D64308A01DC
:100B60009C2064008A11061FAE2D031705308D00EE
:100B700003135E088A018E20031709308D000313CA
:100B800058088A018E2003170A308D0003135A0873
:100B90008A018E2003170B308D0003135C088A0135
:100BA0008E2007138316071383120712831607126A
:100BB000831287118316871183128512831685127B
:100BC0008312E00A0319E10A6008A0006108A1008D
:100BD0008C30A300A0308A01BF208A11031DC92FC9
:100BE0008A0193213C08A6003D08A7007D30A200A1
:100BF000A3018A01F120B2002508B3003208A00049
:100C00003308A100A2010130A3008A01D520BE0053
:100C10002108BF008A019D214208A6004308A700C1
:100C20007D30A200A3018A01F120B2002508B300A3
:100C30003208A0003308A100A2010130A3008A01FC
:100C4000D520C4002108C5008A01A7214608A600B6
:100C50004708A7007D30A200A3018A01F120B2005D
:100C60002508B3003208A0003308A100A20101301A
:100C7000A3008A01D520C8002108C9008A01B1213A
:100C80004A08A6004B08A7007D30A200A3018A01F4
:100C9000F120B2002508B3003208A0003308A100FB
:100CA000A2010130A3008A01D520CC002108CD008B
:100CB000FE308A01212001308A01212041308A0141
:100CC00021205F08A5005E088A0103203A308A01CE
:100CD000212042308A0121205908A50058088A01A4
:100CE00003203A308A01212043308A0121205B0809
:100CF000A5005A088A0103203A308A012120443095
:100D00008A0121205D08A5005C088A0103202030AB
:100D10008A01212020308A012120FE308A012120F1
:100D2000C0308A01212062088A0121203F08A500E5
:100D30003E088A01032020308A012120FE308A01EA
:100D40002120C0308A012120FE308A012120143068
:100D50008A012120FE308A01212014308A012120BD
:100D6000FE308A01212014308A0121203A308A0184
:100D7000212063088A0121204508A50044088A0132
:100D8000032020308A012120FE308A012120C0303A
:100D90008A012120FE308A01212014308A0121207D
:100DA000FE308A01212014308A012120FE308A0180
:100DB000212014308A012120FE308A0121201430A4
:100DC0008A012120FE308A01212014308A0121204D
:100DD000FE308A01212014308A012120FE308A0150
:100DE000212014308A0121203A308A012120640810
:100DF0008A0121204908A50048088A0103202030E3
:100E00008A012120FE308A012120C0308A01212060
:100E1000FE308A01212014308A012120FE308A010F
:100E2000212014308A012120FE308A012120143033
:100E30008A012120FE308A01212014308A012120DC
:100E4000FE308A01212014308A012120FE308A01DF
:100E5000212014308A012120FE308A012120143003
:100E60008A012120FE308A01212014308A012120AC
:100E7000FE308A01212014308A012120FE308A01AF
:100E8000212014308A012120FE308A0121201430D3
:100E90008A0121203A308A01212065088A01212017
:100EA0004D08A5004C088A01032020308A0121202A
:100EB00064008A11061FF9293E08A0003F08A1001E
:100EC0005F08A3005E088A01C2208A11031D702FEB
:100ED00007138316071383122D30E2008A11762F31
:100EE00007178316071383122B30E2004408A00073
:100EF0004508A1005908A30058088A01C2208A1198
:100F0000031D8A2F07128316071283122D30E30068
:100F10008A11902F07168316071283122B30E300D5
:100F20004808A0004908A1005B08A3005A088A01EC
:100F3000C2208A11031DA42F8711831687118312E3
:100F40002D30E4008A11AA2F87158316871183128A
:100F50002B30E4004C08A0004D08A1005D08A30060
:100F60005C088A01C2208A11031DBE2F85128316D8
:100F7000851283122D30E5008A11C42F8516831641
:100F8000851283122B30E5005A308A019C208A0199
:100F9000E12D071383160713831207128316071216
:100FA0008312871183168711831285128316851287
:100FB000FE3083128A01212001308A0121204F3026
:100FC0008A01212076308A01212065308A01212082
:100FD00072308A01212020308A01212031308A019B
:100FE000212020308A01212068308A0121206F30A1
:100FF0008A01212075308A01212072308A01212046
:1010000020308A01212021308A012120FE308A01EE
:101010002120C0308A01212048308A0121206530FA
:101020008A01212061308A01212074308A01212027
:1010300020308A0121206F308A01212066308A0108
:10104000212066308A01212020308A01212062304F
:101050008A01212079308A01212020308A01212033
:1010600074308A01212069308A0121206D308A0183
:10107000212065308A01212086138316861383126E
:1010800064008A11061FF9298A15402864308A01F4
:101090009C2064008A15861E4628861383168613B4
:1010A000063083128A018620E80007308A018620F4
:1010B000E70008308A018620C000C10109308A019A
:1010C0008620E6006708A600A701A2010130A30060
:1010D0008A01F120B2002508B30068083207D40065
:1010E00033080318013ED500FE308A01212001306B
:1010F0008A01212053308A01212074308A01212065
:101100006F308A01212070308A01212020308A012D
:10111000212074308A01212065308A0121206D3020
:101120008A01212070308A0121202E308A0121205D
:101130003D308A0121204108A50040088A01032092
:10114000FE308A012120C0308A01212052308A01DC
:1011500021203A308A0121204E308A012120653039
:101160008A01212078308A01212074308A012120CF
:1011700020308A01212059308A0121203A308A0109
:10118000212044308A0121206E308A012120203024
:101190008A01212042308A0121203A308A0121200F
:1011A00055308A01212070308A01212096308A0131
:1011B0009C2064008A15061EE72864008A15861E96
:1011C000FA2864008A15061F10298A15D928C00A32
:1011D0000319C10A4008A0004108A100A3015A3028
:1011E0008A01C2208A15031DF8285A30C000C101A7
:1011F0008A1574280130C0020030031C013EC10270
:101200004008A0004108A100A3010A308A01BF20C4
:101210008A15031D0E290A30C000C1018A157428E1
:1012200064308A019C2064008A15061F1029FE3054
:101230008A01212001308A01212054308A01212095
:1012400069308A0121206D308A01212065308A01B0
:10125000212072308A0121203D308A012120550849
:10126000A50054088A01032030308A012120733000
:101270008A01212065308A01212063308A012120E2
:10128000FE308A012120C0308A01212052308A019B
:1012900021203A308A0121204E308A0121206530F8
:1012A0008A01212078308A01212074308A0121208E
:1012B00020308A01212059308A0121203A308A01C8
:1012C000212044308A0121206E308A0121202030E3
:1012D0008A01212042308A0121203A308A012120CE
:1012E00055308A01212070308A01212096308A01F0
:1012F0009C2064008A15061E872964008A15861EB4
:101300009C2964008A15061FB2298A157929D40AF6
:101310000319D50A5408A0005508A100FD30A30008
:1013200020308A01C2208A15031D9A292030D4005A
:10133000FD30D5008A1517290130D4020030031C76
:10134000013ED5025408A0005508A100A3010130B8
:101350008A01BF208A15031DB0290130D400D501B0
:101360008A15172964308A019C2064008A15061F9B
:10137000B229FE308A01212001308A0121204C301F
:101380008A0121206F308A01212077308A012120B3
:1013900065308A01212072308A01212044308A017F
:1013A000212075308A01212074308A012120793072
:1013B0008A0121203D308A01212066088A0102200D
:1013C00025308A012120FE308A012120C0308A0187
:1013D000212052308A0121203A308A0121204E30CA
:1013E0008A01212078308A01212020308A012120A1
:1013F00059308A0121203A308A01212044308A0163
:1014000021206E308A01212020308A0121204230A3
:101410008A0121203A308A01212055308A01212079
:1014200070308A01212096308A019C2064008A1540
:10143000061E242A64008A15861E2F2A64008A1537
:10144000061F3A2A8A15162AE60A64004630660202
:101450008A15031C2D2A4630E6008A15B929E603B1
:101460006400033066028A150318382A0230E60049
:101470008A15B9295408E8005408A0005508A100AD
:10148000A2010130A3008A01D520E700031706302E
:101490008D00031368088A018E20031707308D0022
:1014A000031367088A018E20031708308D00031389
:1014B00040088A018E20031709308D000313660847
:1014C0008A018E20FE308A01212001308A012120EC
:1014D00043308A01212079308A01212063308A013A
:1014E00021206C308A01212069308A01212063305B
:1014F0008A01212061308A0121206C308A0121205B
:1015000020308A01212064308A01212072308A0132
:10151000212065308A01212073308A012120733017
:101520008A01212020308A0121203F308A01212098
:10153000FE308A012120C0308A01212059308A01E1
:1015400021203A308A0121204E308A0121206F303B
:101550008A01212020308A01212042308A01212065
:101560003A308A01212059308A01212065308A01D0
:10157000212073308A01212064008A15861EC62A24
:1015800064008A15061E762B8A15BC2AFE308A0155
:10159000212001308A01212044308A012120753028
:1015A0008A01212074308A01212079308A0121208A
:1015B0003D308A01212066088A01022025308A01F7
:1015C00021203A308A01212043308A0121207530C0
:1015D0008A01212074308A0121203D308A01212096
:1015E0004108A50040088A01032063308A012120B8
:1015F0008A01BB218617831686138312D201D30179
:101600005208A0005308A100B630A3006C308A0134
:10161000BF208A15031D332B0717831607130310EA
:101620008312660DB200B301B30D3308A100320876
:101630008A01AA2007138316071383126608643CE5
:10164000B2000030031CFF3EB3000310B20DB30D17
:101650003308A10032088A01AA20D20A0319D30A4A
:101660008A15031D002B03308A017120BC0021085C
:10167000BD003C08A6003D08A7007D30A200A301E4
:101680008A01F120B2002508B3003208A000330817
:10169000A100A2010130A3008A01D520BE002108CB
:1016A000BF000130D4020030031C013ED5028A0184
:1016B000BB2164008A11061FF9295408A0005508AF
:1016C000A100A30100308A01B9208A15031DAD2CA9
:1016D0003E08A0003F08A1004108A30040088A017D
:1016E000BC208A15031DD52C8A15FE2AFE308A01DE
:1016F000212001308A01212066088A01022025303C
:101700008A01212074308A0121206F308A01212032
:101710000A306607B200B301B30D3308A5003208E2
:101720008A01032025308A0121203A308A012120B4
:1017300043308A01212075308A01212074308A01CA
:1017400021203D308A0121204108A50040088A015E
:10175000032063308A0121208A01BB21861783166A
:1017600086138312D001D1015008A0005108A100B6
:10177000A30114308A01BF208A15031D0B2CD2014E
:10178000D3015208A0005308A1000430A3007D300B
:101790008A01BF208A15031D052C0717831607131E
:1017A00003108312660DB200B301B30D5008B207E7
:1017B00051080318013EB3073308A10032088A011B
:1017C000AA2007138316071383125008C83CB200DF
:1017D0005108031C013E003CB3000310660DB40029
:1017E000B501B50D34083202B4003508031C013EC2
:1017F0003302B5003508A10034088A01AA20D20AB4
:101800000319D30A8A15031DC12BD00A0319D10A63
:101810008A15031DB42B8613831686138312133087
:10182000D000D1015008A0005108A100A30101304F
:101830008A01C2208A15031D6A2CD201D3015208E5
:10184000A0005308A1000430A3007C308A01BF200F
:101850008A15031D632C07178316071303108312C1
:10186000660DB200B301B30D5008B207510803185A
:10187000013EB3073308A10032088A01AA200713EA
:101880008316071383125008C83CB2005108031C8A
:10189000013E003CB3000310660DB400B501B50D68
:1018A00034083202B4003508031C013E3302B5008F
:1018B0003508A10034088A01AA20D20A0319D30AE4
:1018C0008A15031D1F2C0130D002031CD1028A157A
:1018D0000318122C03308A017120BC002108BD00BE
:1018E0003C08A6003D08A7007D30A200A3018A01A4
:1018F000F120B2002508B3003208A0003308A1008F
:10190000A2010130A3008A01D520BE002108BF003A
:101910000130D4020030031C013ED5028A01BB21F4
:1019200064008A11061FF9295408A0005508A10077
:10193000A30100308A01B9208A15031DAD2C3E0891
:10194000A0003F08A1004108A30040088A01BC2074
:101950008A15031DD52C8A15AE2B07138316071382
:101960008312861383168613FE3083128A01212088
:1019700001308A01212046308A01212069308A0104
:1019800021206E308A01212069308A0121207330A4
:101990008A01212068308A01212020308A012120FB
:1019A00021308A0121208A15402886138316861348
:1019B000FE3083128A01212001308A0121204F301C
:1019C0008A01212076308A01212065308A01212078
:1019D00072308A01212020308A01212074308A014E
:1019E000212065308A0121206D308A01212070304C
:1019F0008A0121202E308A01212021308A012120D4
:0A1A00008A15402863008A15022DA4
:02400E00723D01
:0E420A001E001200000032001E001E001E00EA
:00000001FF
